:020000040000FA
:0600000044EF02F01200C3
:02002A000000D4
:04002C00300E066E1E
:10003000750E076E0606000E075A0650071003E0FD
:1000400000000000F7D727D803000000C950036E56
:10005000F292D66AF2940A6A0B6A090E0A5C000EE2
:100060000B5816E29E969E50080B04E1F250040BCA
:1000700001E1F9D7F2B40CD0100E0A24E96E000E9B
:100080000B20EA6EC9CFEFFF0A2A000E0B22E5D73C
:1000900048D8DAD71200720ED36E0F015A690F01D9
:1000A0005B690F015C690F015D690F018B0E596F70
:1000B0000F01360E586F600E0E6E0F0E0F6E056A32
:1000C0001C0E055C0AE20EC0E9FF0FC0EAFF0E2A13
:1000D000000E0F22EF6A052AF3D7100E7A6E3F0E3C
:1000E000C16E926A010E936E180E946E806A816AD8
:1000F000826A350EC66EC76AC30ED56EF19CF29247
:10010000F288026A300E066E750E076E0606000E45
:10011000075A0650071003E000000000F7D7D09CF4
:100120001200056A046A0A50055C000E0B5418E2BE
:100130000550EA6A100FE96E000EEA22EF50036ED6
:100140000528EA6A100FE96E000EEA22EF502E0829
:1001500003E1010E026E052A04D8052A042AE3D71A
:1001600012000350F66EF76AD890F636F736EA0EAC
:10017000F626020EF7220900F5CF00F00A00F5CFAF
:1001800001F00450FE0BE8420D6A600F0C6E0F0E7A
:100190000D22025002E00088026A0450010B49E17E
:1001A00001500F0B0CC0E9FF0DC0EAFFE8500F0B28
:1001B000F36EF00EEF14F310EF6E0150F00BE84207
:1001C000E842E842E8421C6E0CC0E9FF0DC0EAFFBD
:1001D000060EE926000EEA221C500F0BF36EF00EFD
:1001E000EF14F310EF6E00500F0B1C6E0CC0E9FF04
:1001F0000DC0EAFF110EE926000EEA221C500F0B7B
:10020000F36EF00EEF14F310EF6E0050F00BE842B7
:10021000E842E842E8421C6E0CC0E9FF0DC0EAFF6C
:10022000170EE926000EEA221C500F0BF36EF00E9B
:1002300058D001500F0B0CC0E9FF0DC0EAFFE85089
:100240000F0BF36EF346F346F346F3460F0EEF142F
:10025000F310EF6E0150F00BE842E842E842E8424A
:100260001C6E0CC0E9FF0DC0EAFF060EE926000E69
:10027000EA221C500F0BF36EF346F346F346F346A7
:100280000F0EEF14F310EF6E00500F0B1C6E0CC02E
:10029000E9FF0DC0EAFF110EE926000EEA221C500C
:1002A0000F0BF36EF346F346F346F3460F0EEF14CF
:1002B000F310EF6E0050F00BE842E842E842E842EB
:1002C0001C6E0CC0E9FF0DC0EAFF170EE926000EF8
:1002D000EA221C500F0BF36EF346F346F346F34647
:0A02E0000F0EEF14F310EF6E120082
:0602EA00000100100100FC
:1002F00020000200002000400004000800800800E8
:1003000080004000040000021000FFFFDCCEFFFF71
:10031000FFFFFFFFFFFFFFFFFFFFFFFFFFFFFFFFED
:10032000FFFFFFFFFFFFFFFFFFFF0000FFFFFFFFDB
:100330008004FFFFFFFFFFFF0002808004048CC4E5
:1003400048480000084037B1048027B101102A5105
:100350002911097029612B6140812B71297137B1F5
:1003600000008080284004040871FFFF0B716919A8
:1003700022216119226102612B210B706009231077
:1003800082E0222003B4833423310A71A3318A71BD
:1003900029614009233006A0873084844084248169
:1003A000FFFFFFFFFFFF8400FFFFFFFF0B716919D5
:1003B00022216119226102612B210B706009231037
:1003C00082E0222003B4833423310A71A3318A717D
:1003D00029614009233006A0873084844084248129
:0A03E000FFFFFFFFFFFFFFFFFFFF1D
:0603EA002A0EF66E000E63
:1003F000F76E000EF86E00010900F550656F0900F8
:10040000F550666F03E1656701D03DD00900F550F6
:10041000606F0900F550616F0900F550626F0900C7
:100420000900F550E96E0900F550EA6E090009006F
:100430000900F550636F0900F550646F0900090069
:10044000F6CF67F0F7CF68F0F8CF69F060C0F6FF3D
:1004500061C0F7FF62C0F8FF0001635302E164531B
:1004600007E00900F550EE6E6307F8E26407F9D77C
:1004700067C0F6FF68C0F7FF69C0F8FF00016507B5
:08048000000E665BBFD71200FD
:0804880012EE00F022EE00F07C
:10049000F86A1B9CF5EC01F059EC02F016EC00F048
:0404A000FBD7120074
:0C04A40000EE00F00F0EEE6AEA62FDD7D9
:0204B000120038
:0204B200120036
:020000040030CA
:0100010009F5
:010002001AE3
:010003001EDE
:010005008179
:010006008178
:0100080001F6
:00000001FF
